:020000040000FA
:060000000A30A6001A28D8
:080008000B11A4000308831290
:100010000313A500A60B15288619122886150A3089
:10002000A600152886110A30A60025088300A40E14
:10003000240E090083160313003085000230860069
:10004000D7308100CF3099000030980004309F00F5
:100050008312031307309F008B178B1600309A0012
:10006000903098008C1E32281A08A000A700A70E16
:10007000F039A0002708F03903112002031D3228AF
:100080008316031300308600831203130030980098
:1000900003112008903C03194E285428200886009C
:1000A0000514572005105628200886001A28063007
:1000B000A100DA30A200FF30A300A30B5D28A20B41
:0800C0005B28A10B5928080080
:02400E00293F48
:00000001FF
